:030000000245F2C4
:0C45F20078FFE4F6D8FD758161024639BF
:101DD5000A53746172743A20004950436F6E6E6500
:101DE50063745245510A004950436F6E6E656374C2
:101DF500003E432C562C43432CC0E4E0EFF2E5F0C3
:101E050020D1E8EDEAEEEC49500A003E432C4D4165
:101E1500432C25303262583A25303262583A253003
:101E25003262583A25303262583A25303262583A91
:101E350025303262582C4D414320E0E4F0E5F10AAB
:101E4500003E432C5645522C20332E3120EEF220F5
:101E550025732025732CC2E5F0F1E8FF20495020B9
:101E6500ECEEE4F3EBFF0A004E6F762030332032C0
:101E75003030370030383A35303A3536003E432C6D
:101E85004C442C50524F473A20202020202020201F
:101E9500202020202020202020202020202020203D
:101EA500202020202020202020202020202020202D
:101EB500202020202020202020202020202020201D
:101EC500202020202020202020202020202CC4E09D
:101ED500F2E020EFF0EEF8E8E2EAE828F4E0E9EBDA
:101EE500290A003E2A2C312CCEF1EDEEE2EDFBE580
:101EF50020EFE0F0E0ECE5F2F0FB20F1E5F2E5E2C1
:101F0500EEE3EE20E8EDF2E5F0F4E5E9F1E00A00B4
:101F15003E412C4130312C2562752E2562752E25CA
:101F250062752E2562752C495020E0E4F0E5F1201C
:101F3500E0E4E0EFF2E5F0E00A003E412C4130320A
:101F45002C2562752E2562752E2562752E256275E6
:101F55002C495020E0E4F0E5F120EEF1ED2E20F1E2
:101F6500E5F0E2E5F0E00A003E412C4130332C2556
:101F750062752E2562752E2562752E2562752C4992
:101F85005020E0E4F0E5F120F0E5E72E20F1E5F062
:101F9500E2E5F0E00A003E412C4130342C25627523
:101FA5002E2562752E2562752E2562752CCCE0F1E5
:101FB500EAE020F1E5F2E80A003E412C4130352CFB
:101FC5002562752E2562752E2562752E2562752C66
:101FD500D8EBFEE70A003E532C4130362C256275BE
:101FE5002CC2F0E5ECFF20EEE6E8E42E20EAE2E87C
:101FF500F2E0EDF6E8E820282A3130ECF1290A0074
:102005003E2A2C312CC4EEEF2E20EFE0F0E0ECE57B
:10201500F2F0FB20F1E5F2E5E2EEE3EE20E8EDF289
:10202500E5F0F4E5E9F1E00A003E422C5330312CAD
:102035002562752CC6E4E0F2FC20E7E0EFF0EEF156
:10204500E020F1EEE5E4E8EDE5EDE8FF20EEF22035
:10205500F1E5F0E2E5F0E00A003E422C5330322C87
:102065002562752CCEE1ECE5ED20F120F1E5F0E2FD
:10207500E5F0EEEC20E1E5E720EAE2E8F2E0EDF656
:10208500E8E90A003E422C5330332C2562752CCFEB
:10209500E5F0E5E7E0EFF3F1EA20EFF0E820EFEE19
:1020A500F2E5F0E520F1E2FFE7E820F120F1E5F0C7
:1020B500E2E5F0EEEC0A003E422C5330342C25626A
:1020C500752CCDE5F220EFE5F0E5E4E0F7E820E456
:1020D500E8E0E3EDEEF1F2E8EAE820E220F1E5F0F0
:1020E500E2E5F00A003E422C5330352C2562752C72
:1020F500CAE0EDE0EB20F8E8F0EEEAEEE2E5F8E024
:10210500F2E5EBFCEDEEE3EE20EEE1ECE5EDE00AC9
:10211500003E532C5330362C253032625825303250
:102125006258253032625825303262582530326285
:102135005825303262582C4D414320E0E4F0E5F15A
:1021450020F8E8F0EEEAEEE2E5F8E0F2E5EBFCED8A
:10215500EEE3EE20EEE1ECE5EDE00A003E454E440F
:102165000A0044756D705820202020203030203022
:102175003120303220303320303420303520303695
:10218500203037203038203039203041203042206F
:1021950030432030442030452030460A003A2000A4
:1021A5000A0044756D7044202020202030302030F6
:1021B5003120303220303320303420303520303655
:1021C500203037203038203039203041203042202F
:1021D50030432030442030452030460A0045727295
:1021E500206B657900526420656570726F6D0A0019
:1021F5005264204D454D0A00526420436F64650AC0
:102205000044656275674950204F4E0A0044656277
:1022150075674950204F46460A0044656275675503
:10222500736572204F6E0A00446562756755736564
:1022350072204F46460A0044656275674D736720F4
:102245004F6E0A0044656275674D7367204F4646B9
:102255000A00436F6E666967206C6F636B210A0025
:10226500577220656570726F6D0A0020536176653F
:1022750020656570726F6D210A00457272204D41AF
:102285004321004C6F61643E3E002A003C413031E1
:102295003D003C4130323D003C4130333D003C4146
:1022A50030343D003C4130353D003C4130363D0049
:1022B5004E4F4950004C494E4B434F4E54520054DB
:1022C50052415353004652004E4F4C494E4B004924
:1022D5004E49004E4F4449414700003C21003C53C4
:1022E50030313D003C5330323D003C5330333D00EE
:1022F5003C5330343D003C5330353D003C53303683
:102305003D00FF22B5FF22BAFF22C4FF22CAFF22E9
:0A231500CDFF22D4FF22D8FF22DF03
:06502F00015E00015C00BF
:104FC600C2AFC28E438910758BFF758DB7D2ABD237
:044FD6008ED2AF22A6
:03001B000244316B
:10443100C0E0C083C082C0D0C2AFC28E758BFF7591
:104441008DB720160675A61E75A6E1055CD212E58C
:104451005E6002055EE55DD394014002155D056174
:10446100E561540F7050D21DE561543F701AD210AE
:10447100906EC7E0601204F0E0D394B4400A9080DB
:10448100007480F0C2AF80FE906EC2E0600204F062
:1044910090693EE0600214F0906EC8E0D394014050
:1044A10003E014F0301502055FE560D39464400425
:1044B100D21680020560E55BD394014002155BD200
:0C44C1008ED2AFD0D0D082D083D0E032B9
:1017B400C291C290D2B5C21A7D027C007F07124F3B
:1017C4005A8F26E526646060097D017F60124F12FE
:1017D400D21AE4FDFC7F0B124F5A8F26E52630E621
:1017E400097D04E4FF124F36D21A7D017C007F0785
:1017F400124F5A8F26E5267008FD7FFF124F12D232
:101804001A301A03126000C2AFC288C2A8C2AA75F5
:101814008900124887906B7BE0B4FA09A3E064CE98
:1018240070030218B4E4F52674732526F582E434B3
:101834006BF583E4F00526E526B443EC906B7B74EA
:10184400FAF0A374CEF0A374CCF0906B81740AF018
:10185400E4A3F0A304F0A3F0906B867403F0A374E4
:10186400CCF0906B7774FFF0A3F0A3F0E4A3F090B6
:101874006B927405F0E4F526E5262401FFE433FEBB
:1018840074732526F582E4346BF583E0FD124FADC5
:101894000526E526C3944340DFE4F5A775A61E7527
:1018A400A6E1907FF0F0A3F09080007480F080FEB9
:1018B400D2AF906B867403F0A374CCF0E4906B8584
:1018C400F0123F60EF60031230B0C2B5123455C25B
:1018D40016124C5B906B92E0C3940350037403F0B4
:1018E400D21AC21CC21BD293201A077E1D7FD512A6
:1018F4004046E4906DB2F0124FC6C2AFA37408F034
:10190400906AF17424F0E4A3F0906B7BE0906AF3A6
:10191400F0906B7CE0906AF4F0906B7DE0906AF557
:10192400F0906B7EE0906AF6F0906B7FE0906AF73F
:10193400F0906B80E0906AF8F0755D01E4906DB40E
:10194400F0C217C218D2AF75A70775A61E75A6E117
:10195400124EEB201A19AF267E007D03124127E4B4
:10196400FF1243877E6B7FB2E4FB7D01124201903C
:101974006EC7E060037401F0E490693EF0A374550F
:10198400F0A37481F0E4F55FE4F56090693EE070E3
:1019940003122941906EC8E0B401119080007410C4
:1019A400F0E4906EC8F0D21AD21BD21C908008E0EA
:1019B400F52630E405D2177410F0E52630E508D298
:1019C400199080087420F0E52630E608D21890803B
:1019D400087440F0E55FD394034023908002E4F060
:1019E400908001F0908000F0E55FD39406400FE40E
:1019F400F55FC213906DB4F0755D01124C5B90807D
:101A0400A0E070031249809080B8E070031249FA94
:101A14009080D0E07003124AD9908000E0701330B7
:101A24001710123E5C906B6EEFF0D39400400312DB
:101A340008E7908002E07006908000E06005D2150F
:101A440002198CC215E4F55F90693EE06003021947
:101A54008C301912123A85906B6EEFF0D3940040DB
:101A640005E0FF125002201803021BEB1237A1906D
:101A74006B6EEFF0700302198C906BB2E054BF24CC
:101A84007F7003021B4E147003021B2624026003A2
:101A9400021B81201A077E1D7FDE124046301E790C
:101AA400201376906B8AE07006906B8EE0605B90FA
:101AB4006EBEE0FF906B8AE0B50724906EBFE0FE37
:101AC400906B8BE0B50618906EC0E0FE906B8CE0D6
:101AD400B5060C906EC1E0FE906B8DE06E602B90AD
:101AE4006B8EE06F7033906EBFE0FF906B8FE0B54C
:101AF4000727906EC0E0FF906B90E0B5071B906ED7
:101B0400C1E0FF906B91E0B5070F906DB47401F0E4
:101B1400120021755D01021BEB906EBE74FFF00292
:101B24001BEB906EC7E060037401F0906EB6E0FFAB
:101B3400906BB4E06F6003021BEB906EB6E004F0B0
:101B4400E4F55D906DB2F0021BEB301303021BEB66
:101B5400906B81E0700302198C125036D213E4F5B5
:101B64005D906DB2F0906EC204F0E4906EB5F0A397
:101B7400F0201A737E1D7FEC124046806A906EC777
:101B8400E060037401F0301352906BB2E020E74B35
:101B9400906BB4E0FF906EB5E0FE6F600D906EBD8B
:101BA400E07007EE146F703F8013906EB5E004F0A0
:101BB400906B6EE0FFD394044003124D4290683A58
:101BC4007482F0A37401F0906BB4E090683CF07EF2
:101BD400687F3A7D0312490502198C301E092013CF
:101BE40006906EBE74FFF0201303021CA0E55D7026
:101BF4006B124E33EF60207E6C7FB2906CB3E024A6
:101C040004FD124905906EBDE0600302198C906BCF
:101C140092E0F55D02198C906EC2E0D3943C403C96
:101C2400906EBDE07036906EC204F0906AF0E07081
:101C34002B12501CE4906CB2F0A37412F0906EB6A8
:101C4400E0906CB4F0A374FDF090694163A201903C
:101C54006CB663A2017F1212337E809B125011EF87
:101C6400601590683A7483F0E4A3F07E687F3A7D4F
:101C74000212490502198CE55D6401600302198CA6
:101C8400906DB2E004F0E0C394055003021BFBC264
:101C940013E4906DB4F012002102198CE55D640127
:101CA400600302198C906DB4E014604024FE603C23
:101CB400147003021D882404600302198CE4F55F88
:101CC400201E13906DB47404F0906DB2E05401F0D2
:101CD400755D0102198CE4906DB4F0906DB204F05E
:101CE400755DC8906EBE74FFF002198C906EBEE0F4
:101CF4007003021D77906CB27480F0906CB4740120
:101D0400F0E4A3F0A304F0A37430F0A3747BF0E434
:101D1400F52674B92526F582E4346CF583747DF0D8
:101D240074BA2526F582E4346CF583E4F0E52624C0
:101D340007906CB3F07C6E7DBE906B86E0FAA3E0F6
:101D4400FB7F021247037E6C7FB2E5262409FD1255
:101D54004905906EBDE0601B125036D213E4F55D68
:101D6400906DB2F0906EC204F0E4906EB5F0A3F002
:101D740002198C906DB47404F0906B92E02432F5E7
:101D84005D02198C9080027410F0755D03906DB241
:101D9400E06401FFF0906DB47401F0EF7019906B82
:101DA4008EE06013FCA3E0FDA3E0FEA3E0FF906ED1
:101DB400BE12280302198C906B8AE0FCA3E0FDA3F9
:101DC400E0FEA3E0FF906EBE12280302198C80FE91
:011DD40022EC
:1008E700906BB3E0B444047F0180027F00906BB249
:1008F700E0B447047E0180027E00EE5F604A906BA1
:100907007BE0906BB4F0906B7CE0906BB5F0906BF4
:100917007DE0906BB6F0906B7EE0906BB7F0906BDC
:100927007FE0906BB8F0906B80E0906BB9F0906BC4
:10093700B37452F0906AEA63A2019080A863A2019F
:100947007F0612337E021138906B6EE0C394085015
:1009570003021141906B7BE0FF906BB4E06F600383
:10096700021141906B7CE0FF906BB5E06F60030272
:100977001141906B7DE0FF906BB6E06F6003021151
:1009870041906B7EE0FF906BB7E06F60030211410F
:10099700906B7FE0FF906BB8E06F600302114190AE
:1009A7006B80E0FF906BB9E06F6003021141906BC1
:1009B700B3E0B44415906AEAE0B4FF0E63A2019075
:1009C70080A863A2017F0612337E906EC7E06003A2
:1009D7007401F0906EC87464F0906BB37452F09029
:1009E7006BB2E0646D6003020B647BFF7A1D79F6DE
:1009F7001223817BFF7A1E7910906B7BE0F52FA382
:100A0700E0F530A3E0F531A3E0F532A3E0F533A339
:100A1700E0F534122381752FFF75301E75316D7522
:100A270032FF75331E7534797BFF7A1E79461223A0
:100A3700817BFF7A1E79821223817BFF7A1E79E8F8
:100A47001223817BFF7A1F7915906B81E0F52FA325
:100A5700E0F530A3E0F531A3E0F5321223817BFF07
:100A67007A1F793F906B8AE0F52FA3E0F530A3E07A
:100A7700F531A3E0F5321223817BFF7A1F796D9060
:100A87006B8EE0F52FA3E0F530A3E0F531A3E0F599
:100A9700321223817BFF7A1F799B906B77E0F52FCA
:100AA700A3E0F530A3E0F531A3E0F5321223817B13
:100AB700FF7A1F79BE906B73E0F52FA3E0F530A3A3
:100AC700E0F531A3E0F5321223817BFF7A1F79DB52
:100AD700906B92E0F52F1223817BFF7A2079051224
:100AE70023817BFF7A20792EA21EE433F52F122370
:100AF700817BFF7A20795E906EBDE0F52F1223810E
:100B07007BFF7A207989906EC7E0F52F1223817BCE
:100B1700FF7A2079BC906AF0E0F52F1223817BFFE2
:100B27007A2079EAA211E433F52F1223817BFF7A29
:100B3700217916906EB7E0F52FA3E0F530A3E0F525
:100B470031A3E0F532A3E0F533A3E0F534122381B6
:100B5700123D437BFF7A21796112238122906BB288
:100B6700E0644C70527E217F67124046906BBAE07A
:100B7700F527A3E0F528E4F5297D03AF28AE271272
:100B870041277E217FA2124046AE27AF28E4FB7D96
:100B9700101242017E217FA512404674102528F5C8
:100BA70028E43527F5270529E529C3941040CA7E8F
:100BB700217FA512404622906BB2E0646C705CF511
:100BC7002B7E217FA7124046E4F52AAF2B7E007DBE
:100BD700031241277E217FA2124046E4F529A82B64
:100BE700E6FF74BC2529F582E4346BF583EFF00545
:100BF7002B0529E529B410E67E6B7FBCE4FB7D104D
:100C07001242017E217FA5124046052AE52AC39498
:100C17000840B87E217FA512404622906BB2E0645F
:100C27004B7061F52974A42529F582E4346BF583AB
:100C3700E0603274A42529F582E4346BF583E0F48F
:100C4700602374A42529F582E4346BF583E0FF74EF
:100C5700BA2529F582E4346BF583E0B50710052939
:100C6700E529B408C090693E7432F0021138906BE0
:100C7700B27421F0301A030211387E217FE212404C
:100C870046021138906BB2E0B4521A201A077E213F
:100C97007FEA124046906BB27472F07E6B7FB27D32
:100CA7000812478722906BB2E064497045201A0703
:100CB7007E217FF5124046906BBAE0F527A3E0F559
:100CC70028E4F529852882852783E0FF74BC252938
:100CD700F582E4346BF583EFF00528E5287002050B
:100CE700270529E529B480DC7E6B7FB27D8A124710
:100CF7008722906BB2E064437079A3E06452704638
:100D0700201A077E217FFD124046906BBAE0F52737
:100D1700A3E0F528E4F529852882852783E493FF56
:100D270074BC2529F582E4346BF583EFF00528E5DB
:100D370028700205270529E529B480DB7E6B7FB281
:100D47007D8A12478722906BB3E0645760030211D4
:100D570041906BBAE0F527A3E0F52874BC2529F587
:100D670082E4346BAD82FC7B80AF28AE27124DFF47
:100D7700021138906BB2E064446003020E0B906B73
:100D8700BAE0FF64447003021138EFB4310CC21AA1
:100D97007E227F06124046021138906BBAE0B430CB
:100DA7000CD21A7E227F12124046021138906BBA7B
:100DB700E0B4320CD21B7E227F1F1240460211384C
:100DC700906BBAE0B4330CC21B7E227F2D124046D3
:100DD700021138906BBAE0B4340CD21C7E227F3CEF
:100DE700124046021138906BBAE0B4350CC21C7E33
:100DF700227F49124046021138906BBAE0FF120079
:100E07001E02113890693EE07013201A077E227F78
:100E170057124046906BB27421F002113890693E28
:100E27007432F0906BB2E0FFB4510A908000748086
:100E3700F0C2AF80FEEF64577045201A077E227F0D
:100E470065124046906BBBE0906B6EF0E4F529901D
:100E57006B6EE0FFE529C39F400302113874BC2580
:100E670029F582E4346BF583E0FF906BBAE025291E
:100E770024E9F582E43469F583EFF0052980D09001
:100E87006BB2E064536003020F3A201A077E227F99
:100E970070124046906B7BE0FF9069F2E06F703C08
:100EA700906B7CE0FF9069F3E06F7030906B7DE0B2
:100EB700FF9069F4E0B50724906B7EE0FF9069F539
:100EC700E0B50718906B7FE0FF9069F6E0B5070C77
:100ED700906B80E0FF9069F7E06F6016906BB274DB
:100EE70021F0301A030211387E227F7F124046021A
:100EF7001138E4F529E4F560AF29FE74E92529F5F1
:100F070082E43469F583E0FD124FAD0529E529C375
:100F170094FE40E19080007480F0C2AFE4907FF0CF
:100F2700F0A3F0907FFD74AAF0A374FFF0A37455AB
:100F3700F080FE906BB2E0644F704C906BBAE0F5B6
:100F470027A3E0F528E5284527700A201A077E22FF
:100F57007F88124046201A077E227F8F124046E480
:100F6700F52974BC2529F582E4346BF583E08528DF
:100F770082852783F00528E528700205270529E5DE
:100F870029B480DE021138906BB2E0FFB445279098
:100F970080007480F0906BBAE0FDA3E0907FF0CD05
:100FA700F0A3EDF0C2AF907FFD74AAF0A374FFF039
:100FB700A37455F080FEEF64656003021138906BEF
:100FC700BAE0FFA3E0907FF0CFF0A3EFF0E4F527BE
:100FD700F528D3907FF1E09528907FF0E0952740A2
:100FE70020E4F5602528FFE5273401FE8528828562
:100FF7002783E0FD124FAD0528E5287002052780FD
:10100700D17E227F9112467EEF4E60201200039020
:101017006B81EFF0120003906B82EFF012000390E8
:101027006B83EFF0120003906B84EFF07E227F97C3
:1010370012467EEF4E6020120003906B8AEFF0128B
:101047000003906B8BEFF0120003906B8CEFF012A4
:101057000003906B8DEFF07E227F9D12467EEF4E50
:101067006020120003906B8EEFF0120003906B8FDD
:10107700EFF0120003906B90EFF0120003906B916A
:10108700EFF07E227FA312467EEF4E602012000310
:10109700906B77EFF0120003906B78EFF01200037C
:1010A700906B79EFF0120003906B7AEFF07E227F5E
:1010B700A912467EEF4E6020120003906B73EFF08B
:1010C700120003906B74EFF0120003906B75EFF052
:1010D700120003906B76EFF07E227FAF12467EEF11
:1010E7004E6008124BFE906B92EFF0E4F529E4F5A1
:1010F70060E5292401FFE433FE74732529F582E4B2
:10110700346BF583E0FD124FAD0529E529C3944300
:1011170040DC9080007480F0C2AFE4907FF0F0A3D1
:10112700F0907FFD74AAF0A374FFF0A37455F080CC
:0A113700FE7E6B7FB27D0812478731
:01114100228B
:104DC700AE07EEC39430400BEED394395005EE2472
:104DD700D0FF22EEC39461400BEED394665005EEEC
:104DE70024A9FF22EEC39441400BEED3944650050D
:084DF700EE24C9FF22AF0622E1
:104F9300906AE9E004F07006906AE8E004F0906A31
:0A4FA300E8E0FEA3E0FF124F7722C2
:10000300124F93124DC7EFC454F0FEC006124F9324
:08001300124DC7D0E02FFF22BF
:104BFE00E4907003F0124F93907004EFF0C3943072
:104C0E004018E0FFD394395011907003E02441F521
:104C1E0082E43469F583EFF08011907003E0244153
:104C2E00F582E43469F583E4F0800C907003E004BF
:104C3E00F0E0D3940840BE75320075330075340031
:0C4C4E00E4F5357B017A6979411235FDEF
:014C5A002237
:04467E008E2C8F2DC2
:10468200906AE8E4F0A374FFF0124F93EF606EF4C7
:10469200606B852D82852C83E493B507EC752E0122
:1046A200E52D252EF582E4352CF583E493602590E3
:1046B2006AE9E0252EFF906AE8E03400FE124F77A7
:1046C200E52D252EF582E4352CF583E493B5070418
:1046D200052E80CCE52D252EF582E4352CF583E4DC
:1046E2009370A6E52E24FFFFE434FFFE906AE9E012
:1046F2002FF0906AE8E03EF07E007F0122E4FEFFA8
:014702002294
:103F60007E227FE012467EEF4E70037F01227E228A
:103F70007FE312467EEF4E600C124F93EF24D02465
:103F8000FF921E8002D21E7E227FE912467EEF4EF5
:103F9000600C124F93EF24D0906EBDF08005E4903A
:103FA0006EBDF07E227FEF12467EEF4E600C124F08
:103FB00093EF24D0906EC7F08005E4906EC7F07E3A
:103FC000227FF512467EEF4E600C124F93EF24D005
:103FD000906AF0F08005E4906AF0F07E227FFB1298
:103FE000467EEF4E600C124F93EF24D024FF9211C7
:103FF0008002C211906B7B63A201906EB763A20135
:104000007F0612337E30113B7E237F0112467EEF06
:104010004E6030120003906EB7EFF0120003906E06
:10402000B8EFF0120003906EB9EFF0120003906E3B
:10403000BAEFF0120003906EBBEFF0120003906E27
:06404000BCEFF07F00223E
:1030B000C211E4906EC7F0D21EC214906EBDF090A3
:1030C0006AF0F0906B7B63A201906EB763A2017F00
:1030D0000612337EE4F527E52775F003A42407F5EF
:1030E00082E43423F583E493FB740193FA7402932E
:1030F000F912267B70030232A2E4F528F529FD744B
:10310000692DF582E43469F583E0FF700302329D96
:10311000E52775F003A42407F582E43423F583E45E
:1031200093FB740193FA740293F9852882758300E6
:10313000122694FEEFB5060875290105280232997A
:10314000E5297003023299EE6003023294E52724E8
:10315000FE602814700302327C1470030232801463
:10316000700302328814700302328C24056003025B
:10317000329D906EC77401F002329DD21174692D98
:10318000F582E43469F583E0FF642D700302329D1B
:10319000124DC7EFC454F0FC746A2DF582E4346913
:1031A000F583E0FF124DC7EF2C906EB7F0746B2DD6
:1031B000F582E43469F583E0FF124DC7EFC454F0A3
:1031C000FC746C2DF582E43469F583E0FF124DC781
:1031D000EF2C906EB8F0746D2DF582E43469F583B0
:1031E000E0FF124DC7EFC454F0FC746E2DF582E47D
:1031F0003469F583E0FF124DC7EF2C906EB9F0747F
:103200006F2DF582E43469F583E0FF124DC7EFC4FA
:1032100054F0FC74702DF582E43469F583E0FF12FC
:103220004DC7EF2C906EBAF074712DF582E43469BD
:10323000F583E0FF124DC7EFC454F0FC74722DF516
:1032400082E43469F583E0FF124DC7EF2C906EBB2A
:10325000F074732DF582E43469F583E0FF124DC7F5
:10326000EFC454F0FC74742DF582E43469F583E006
:10327000FF124DC7EF2C906EBCF08021D214801D40
:10328000906EBD7401F08015C21E8011906AF074BA
:1032900001F08009E4F529F5280D0230FF05270229
:0232A00030D725
:0132A2002209
:104CB400906DB3E0C3947C503D906DB3E0FE04F07E
:104CC40074F12EF582E4346AF583EFF0BF0A27907D
:104CD4006DB3E0FF04F074F12FF582E4346AF583D8
:104CE400E4F0906DB3E0FF124809906DB37408F0DE
:074CF400906AF2E004F022D7
:104C5B009080007480F0906B7363A201F583F582F2
:104C6B0063A2017F0812337E906B7B63A20190805D
:104C7B008863A2017F0A12337E908092E4F0A374C2
:104C8B0032F0A37401F0906B85E0FF9080B1F0904F
:104C9B0080E1EFF09080957455F0A3F09080007454
:094CAB0001F09080097470F02200
:10498000908009E04410F09080A0E0706C9080A1CD
:104990007482F09080A874FFF0A3F0A3F0A3F07FDE
:1049A000039080AEEFF07FCBA3EFF07F039080AC5D
:1049B000EFF0A374CBF09080007402F0906FF712C8
:1049C000280F00000000906FF7E0908040F0906F9B
:1049D000F8E0908041F0906FF9E0908042F0906FA5
:1049E000FAE0908043F0A3E4F0A3F0A3F0A3F090EA
:0949F0008018F0A3F0A3F0A3F07D
:0149F900229B
:104AD900908009E04440F09080D17482F0906B8618
:104AE900E0FF9080DEF0906B87E0FF9080DFF09030
:104AF90080027402F0906FFB12280F0000000090F2
:104B09006FFBE0908058F0906FFCE0908059F09036
:104B19006FFDE090805AF0906FFEE090805BF0A30B
:104B2900E4F0A3F0A3F0A3F0908030F0A3F0A3F099
:024B3900A3F0E7
:014B3B002257
:1049FA00908009E04420F09080B8E0706C9080B913
:104A0A007482F07F039080C6EFF07FCDA3EFF07F32
:104A1A00039080C4EFF0A374CDF09080C074FFF0CF
:104A2A00A3F0A3F0A3F09080017402F0906FFF123C
:104A3A00280F00000000906FFBE090804CF0906F10
:104A4A00FCE090804DF0906FFDE090804EF0906F0A
:104A5A00FEE090804FF0A3E4F0A3F0A3F0A3F0905F
:094A6A008024F0A3F0A3F0A3F0F6
:014A73002220
:104703008C278D28A907EAFDE975F018A424ACFFCE
:10471300E5F034808F82F583EDF0EBFDE975F01859
:10472300A4FFAEF024ACFBEE34808B82F583A3EDC3
:10473300F08528828C83E0FDEF24A8FFEE3480FE11
:104743008F82F583EDF08528828C83A3E08F828EA0
:1047530083A3F0852882852783A3A3E0FDE975F071
:1047630018A424A8FFE5F03480FE8F82F583A3A369
:10477300EDF08528828C83A3A3A3E08F828E83A38D
:04478300A3A3F022DA
:064787008D2CAB07AA0611
:10478D00906FF7E0FCA3E0FDA3E0FEA3E0F5308E13
:10479D002F8D2E8C2DAE02AF038E838F8263A201DF
:1047AD00E52F540744C0F58385308263A201AF2CF9
:1047BD001233E7908000E020E5F9E4FCFDFEE530E2
:1047CD00252CF530EE352FF52FED352EF52EEC355C
:1047DD002DF52D908040E52DF0A3E52EF0A3E52FCE
:1047ED00F0A3E530F09080007420F0AF30AE2FAD27
:0B47FD002EAC2D906FF7122803AF2C9C
:01480800228D
:064905008D27AB07AA0696
:10490B00906FFBE0FCA3E0FDA3E0FEA3E0F52B8E94
:10491B002A8D298C28AE02AF038E838F8263A2016E
:10492B00E52A540744D0F583852B8263A201AF2778
:10493B001233E7E4FCFDFEE52B2527F52BEE352A9C
:10494B00F52AED3529F529EC3528F528908058E521
:10495B0028F0A3E529F0A3E52AF0A3E52BF090803E
:10496B00027420F0AF2BAE2AAD29AC28906FFB124E
:04497B002803AF2737
:01497F002215
:024387008F287D
:10438900908001E030E5037F0022906FFFE0FCA3FD
:10439900E0FDA3E0FEA3E0F52C8E2B8D2A8C29905D
:1043A9006EB763A201E52B540744C8F583852C82B7
:1043B90063A2017F061233FDE52C2406F52CE435B2
:1043C9002BF52BE4352AF52AE43529F529906DB525
:1043D90063A201E52B540744C8F583852C8263A2A7
:1043E90001AF281233FDE4FCFDFEE52C2528F52C50
:1043F900EE352BF52BED352AF52AEC3529F52990E3
:10440900804CE529F0A3E52AF0A3E52BF0A3E52CE0
:10441900F09080017420F0AF2CAE2BAD2AAC29901E
:074429006FFF122803AF280A
:014430002269
:103E5C009081E0E0F527052705270527052705278D
:103E6C0005270527052705270527908010E0F52A4B
:103E7C00A3E0F52BA3E0F52CA3E0F52D9081E1E078
:103E8C00F5270527052705270527052705270527D6
:103E9C00052705270527908014E0F52EA3E0F52FC4
:103EAC00A3E0F530A3E0F531E530B52C08E531B5EC
:103EBC002D037F0022E4F527E530540744E0F58319
:103ECC0085318263A201906BB263A2017F08123428
:103EDC0015906BB463A201906AEA63A2017F06128B
:103EEC00337E906BB2E0F528A3E0F529E4F527903A
:103EFC006BB2E0702AA3E024F8F527E530540744B0
:103F0C00E0F58385318274082582F582E43583F5EA
:103F1C008363A201906BB263A201AF27123415AE7A
:103F2C0028E4FCFDE5312529F531E5303EF530ED91
:103F3C00352FF52FEC352EF52E908014E52EF0A3B1
:103F4C00E52FF0A3E530F0A3E531F090800074404C
:033F5C00F0AF279C
:013F5F00223F
:1037A1009081E6E0F5270527052705270527052749
:1037B10005270527052705270527908028E0F52AF5
:1037C100A3E0F52BA3E0F52CA3E0F52D9081E7E034
:1037D100F527052705270527052705270527052798
:1037E10005270527052790802CE0F52EA3E0F52F6E
:1037F100A3E0F530A3E0F531E4F527E530B52C0A77
:10380100E531B52D05C2180238FBE530540744F007
:10381100F58385318263A201906BB263A2017F08B7
:10382100123415906BB2E0F528A3E0F529E529459E
:103831002870099080027410F07F0022906EBEE023
:10384100FFF4602D906BB4E06F7076906EBFE0FF77
:10385100906BB5E06F706A906EC0E0FF906BB6E060
:103861006F705E906EC1E0FF906BB7E06F60228079
:1038710050906BB4E0906EBEF0906BB5E0906EBF6F
:10388100F0906BB6E0906EC0F0906BB7E0906EC1B7
:10389100F0906BB2E0702AA3E024F8F527E53054EC
:1038A1000744F0F58385318274082582F582E43579
:1038B10083F58363A201906BB263A201AF27123437
:1038C10015AE28E4FCFDE5312529F531E5303EF55D
:1038D10030ED352FF52FEC352EF52EAF2DAE2CAD6D
:1038E1002BAC2AAB31AA30A92FA82ED31227F24034
:1038F100099080027410F07F002290802CE52EF058
:10390100A3E52FF0A3E530F0A3E531F09080027438
:0439110040F0AF27AC
:01391500228F
:103A85009081E3E0F5270527052705270527052765
:103A95000527052705270527052790801CE0F52A1A
:103AA500A3E0F52BA3E0F52CA3E0F52D9081E4E050
:103AB500F5270527052705270527052705270527B1
:103AC500052705270527908020E0F52EA3E0F52F93
:103AD500A3E0F530A3E0F531E4F527E530B52C0A90
:103AE500E531B52D05C219023BD0E530540744E850
:103AF500F58385318263A20190683E63A2017F0E42
:103B050012342B90683EE0F528A3E0F5299068462D
:103B1500E0FFF46045906EB7E0FEEF6E706EA3E0D7
:103B2500FF906847E06F7064906EB9E0FF90684859
:103B3500E06F7058906EBAE0FF906849E06F704C86
:103B4500906EBBE0FF90684AE06F7040906EBCE0FD
:103B5500FF90684BE06F60048032D2D990683EE0F8
:103B6500702AA3E024F2F527E530540744E8F583ED
:103B7500853182740E2582F582E43583F58363A24F
:103B85000190683E63A201AF2712342BAE28E4FCF6
:103B9500FDE5312529F531E5303EF530ED352FF5DB
:103BA5002FEC352EF52EAF2DAE2CAD2BAC2AAB312F
:103BB500AA30A92FA82ED31227F25006E5294528A9
:103BC50070099080017410F07F0022908020E52E0E
:103BD500F0A3E52FF0A3E530F0A3E531F0908001E7
:053BE5007440F0AF2761
:013BEA0022B8
:044046008E2D8F2EFE
:10404A00906FF7E0FCA3E0FDA3E0FEA3E0F5348E59
:10405A00338D328C31E534FFE5335407FEE42FF516
:10406A0030EE34C0F52F853082F5837423F00530A5
:10407A00E5307002052F532FC7F582852F83740A06
:10408A00F00530E5307002052F532FC7906B7B6324
:10409A00A201852F8385308263A2017F061233E74E
:1040AA0074062530F530E4352FF52F852D83852EBE
:1040BA008263A201852F8385308263A2011233CBEA
:1040CA00908000E020E5F9E4FCFDFE906FF7E0F84F
:1040DA00A3E0F9A3E0FAA3E02FFFEE3AFEED39FDE3
:1040EA00EC38FCEF2408FFE43EFEE43DFDE43CFC32
:1040FA00906FF7122803906FF7E0908040F0906F6E
:10410A00F8E0908041F0906FF9E0908042F0906F73
:0C411A00FAE0908043F09080007420F0E8
:014126002276
:064201008E2D8F2E8D2F83
:10420700906FF7E0FCA3E0FDA3E0FEA3E0F5358E99
:10421700348D338C32E535FFE5345407FEE42FF552
:1042270031EE34C0F530853182F5837423F00531E2
:10423700E531700205305330C7F582853083EBF0E6
:104247000531E531700205305330C7906B7B63A2AF
:104257000185308385318263A2017F061233E774BB
:10426700062531F531E43530F530852D83852E82ED
:1042770063A20185308385318263A201AF2F123398
:10428700E7908000E020E5F97408252FF52FFFE47B
:10429700FCFDFEE5352FF535EE3534F534ED3533D8
:1042A700F533EC3532F532908040E532F0A3E53353
:1042B700F0A3E534F0A3E535F09080007420F0AF6B
:0D42C70035AE34AD33AC32906FF7122803E2
:0142D40022C7
:024809008F40DE
:10480B00906FF7E0FCA3E0FDA3E0FEA3E0F5448E80
:10481B00438D428C41E544FFE5435407FEE42FFFF3
:10482B00EE34C0906AF163A201F5838F8263A2011B
:10483B00AF401233E7908000E020E5F9E4FCFDFE89
:10484B00E5442540F544EE3543F543ED3542F5425D
:10485B00EC3541F541908040E541F0A3E542F0A3F2
:10486B00E543F0A3E544F09080007420F0AF44AE34
:0B487B0043AD42AC41906FF7122803E0
:01488600220F
:064127008E2C8F2DAB056C
:10412D00906FF7E0FCA3E0FDA3E0FEA3E0F5338E76
:10413D00328D318C30E533FFE5325407FEE42FF537
:10414D002FEE34C0F52E852F82F5837423F0052FC5
:10415D00E52F7002052E532EC7F582852E83EBF0C9
:10416D00052FE52F7002052E906B7B63A201852E26
:10417D0083852F8263A2017F061233E77406252FF4
:10418D00F52FE4352EF52E532EC7E52C852F828580
:10419D002E83F0052FE52F7002052E532EC7F582C5
:1041AD00852E83E52DF0052FE52F7002052E532E5C
:1041BD00C7908000E020E5F9E533240AF533E435B6
:1041CD0032F532E43531F531E43530F5309080405B
:1041DD00E530F0A3E531F0A3E532F0A3E533F0903F
:1041ED0080007420F0AF33AE32AD31AC30906FF74C
:0341FD0012280382
:01420000229B
:104F7700E5D220E0FBC2AF438E2075D2028F828E2E
:0B4F870083E0FFE4F5D2538EDFD2AFD1
:014F920022FC
:104FAD00E5D220E0FBC2AF43D2028F828E83EDF0BB
:094FBD0075D25063D250D2AF222C
:10488700E4FDED2401FFE433FE124F7774732DF539
:1048970082E4346BF583EFF00DBD3FE6E4FDED24D4
:1048A7007FFFE433FE124F7774692DF582E4346994
:1048B700F583EFF074692DF582E43469F583E070D0
:1048C7001B74692DF582E43469F5837420F0746AEA
:1048D7002DF582E43469F583E4F080040DBD80BED4
:1048E700E49069E8F0FDEDFF7E00124F7774E92D43
:0D48F700F582E43469F583EFF00DBDFEE9B4
:014904002290
:024DFF008B2CFB
:104E0100A2AF921FC2AF85A22D53A2FE8E838F82C5
:104E110005A28C838D827409123443E52C53A2FEC2
:104E210043A22012344553A2DF852DA2A21F92AFC7
:014E3100FF81
:014E3200225D
:104F5A00A2AF921FC2AF8C838D82EF12344343A259
:0C4F6A002012344553A2DFA21F92AFFFBB
:014F76002218
:024F12008F27E7
:104F1400A2AF921FC2AFE4F5838D827406123443AC
:104F2400E52743A22012344553A2DFA21F92AF7F8C
:014F3400017B
:014F35002259
:024F36008F27C3
:104F3800A2AF921FC2AFE4F5838D82740A12344384
:104F4800E52743A22012344553A2DFA21F92AF7F68
:014F58000157
:014F59002235
:1032A300A907E7FFA805EF93C3966008403B74FCAA
:1032B3002FFF80F00F08EF93C3966008402B74FB39
:1032C3002FFF80E00F08EF93C3966008401B74FA4A
:1032D3002FFF80D00F08EF93D3966008400B74F94B
:1032E3002FFF80C01F1F1F1F1FEF54FEF80303F79C
:1032F300E893FC08E893FD08E893FE08E893FF22AF
:1033030009E993C39D6008402974FB29F980F109F9
:10331300E993C39E6008401A74FA29F980E209E927
:1033230093D39F6008400B74F929F980D3191919B5
:103333001919E9C313C313FF22740093F8ECC3985C
:103343004024701F740193F8EDC3984019701474EE
:0E3353000293F8EEC398400E7009740393F8CD
:10336100EFC39840037F00227F0122EDF8E6F008C9
:10337100A3DFFA22EDF8E0F608A3DFFA22E0A36367
:10338100A201F0A363A201DFF475A20022E0A3630E
:10339100A201F0A363A201E0A363A201F0A363A2CF
:1033A10001E463A201F0A363A201DFE175A200229F
:1033B100E0A363A2016DFE936CFDEE058393FC1502
:1033C1008363A201DFEA75A200227F00E493A36375
:1033D100A201F00F600CA3E583C2E3F58363A201B0
:1033E10080EA75A20022E0A363A201F0A3E583C2F3
:1033F100E3F58363A201DFEE75A20022E0A363A2DD
:1034010001F0A3E583C2E4D2E3F58363A201DFEC1B
:1034110075A20022E583C2E3F583E0A363A201F074
:10342100A363A201DFEE75A20022E583C2E4D2E329
:10343100F583E0A363A201F0A363A201DFEC75A20F
:103441000022F922C002C004C00612FFF0D006D04B
:0434510004D002227F
:104564000A536572763A004572724C656E210A00F0
:10457400205544502054696D654750530A00200A61
:10458400444154414752414D3A20002043414E207A
:1045940054696D654750530A002054726173735314
:1045A400656E644552520A000ACEF8C4EBE8EDFB8E
:1045B40043414E210A000A45727241647243414EDE
:1045C4003A000A00205265496E69742043414E0A3C
:1045D400002043414E283029203E20544F210A0018
:0E45E40020545520300A0020545520310A0082
:03001E00E4FF22DA
:104EC300C2A9438902758C48758A4875D90475DB74
:104ED3004875DC4875DD4875DE48E4F5E9F5F9D237
:084EE300D9C2DAD28CD2DE2222
:104E9500C2D9906EDDE07013E5E92419F5EB30D742
:104EA50006E5F904F5FB2285F9FB22E5E924C8F5B9
:0E4EB500EB30D706E5F904F5FB2285F9FB2268
:104CFB00C2D9906EDDE0702C302C16E5E92432F52C
:104D0B00EB30D707E5F904F5FB800385F9FBC22CE3
:104D1B0022E5E92405F5EB30D706E5F904F5FB228E
:104D2B0085F9FB22E5E92432F5EB30D706E5F904EA
:074D3B00F5FB2285F9FB22C4
:104EEB00124EC3906EDDE0C394645006124A7412E6
:104EFB004E9512503CD22BE4F556906FF5F0F545DC
:074F0B00F55AC22CF55822F3
:104D4200EF24FCF545201A127E457F641240467E10
:104D52006B7FB6E4FBAD45124201E545D3940D40AD
:104D620010201A077E457F6B124046E4F545D22992
:104D720022906BB663A201906FE563A201AF451268
:054D8200337EC229226E
:0F500200D3EF6480948D5006E55A70028F5A22C6
:1029410020D903022A1E202B03022A1EE55A6052B7
:1029510090683E540FFF7D47123375E5476401705F
:102961001E906846E0B4FF0ED22D201A127E457FDC
:10297100741240468009302D06E4F55A022A1E12CF
:102981004E95124B3C201A077E457F82124046200D
:102991001A0B7E687F3EE4FBAD5A124201E4F55A00
:1029A100807BE5456043906FE9E02405F527D394EA
:1029B1000D4007E4F545D2298063906FE5E5275482
:1029C1000FFF7D47123375E54730E702D22CE5470B
:1029D100B40109302D06E54A64016003124B3C1233
:1029E1004E95E4F545D2298034E557601E906EC9B5
:1029F100540FFF7D47123375E547B40103202D03C2
:102A0100124B3C124E95E4F557801220010C906E4A
:102A1100DDE0C394645003124B9E124E95123BEBC2
:102A21008F27EF7003022AE5124CFBE4F558E547C6
:102A3100B4010CD22D201A077E457F8F124046E546
:102A410059C394C8502D30132AE547B4420DE54AC5
:102A5100B40208906AF0E06401601874DE2559F54B
:102A610082E4346EF583E5272559F5597D47AF2773
:102A710012336C301121E54720E71C906DB57D477D
:102A8100AF2712336CAF27124387EF700A201A0762
:102A91007E457F9D124046E54754817047E527D327
:102AA100940D400C201A3D7E457FAC124046803487
:102AB100E549D394074028201A2A7E457FBA12405F
:102AC100469069417D47AF2712336C7E697F41E4AF
:102AD100FBAD271242017E457FC61240468005AFFD
:102AE10027122C06301D2030101B906EDDE0C394A0
:102AF1006450120558E55894F0400A9080007480A3
:102B0100F0C2AF80FEC21D201203022C00E5566008
:102B110031D39401400415568028906FF5E004F0FC
:102B2100E0D39403400D201A077E457FC81240462A
:102B3100124EEB201A077E457FD5124046E4F5562A
:102B4100D22B302A43E557703F906EC904F0A3742D
:102B510008F0A37480F0A37401F0A37406F0906FE1
:102B6100E0E0906ECEF0906FE1E0906ECFF0906F6C
:102B7100E2E0906ED0F0906FE3E0906ED1F0E4A3CC
:102B8100F0A3F075570BC22A302872906FDEE07007
:102B910035E5577031906EC97442F0A37408F09016
:102BA1006FDFE0906ECBF0906FE4E0906ECCF0A31D
:102BB1007401F0755706201A077E457FE4124046DE
:102BC100906FDEE004F0906FDEE06402702FE55755
:102BD100702B906EC97402F0A37408F0906FDFE05F
:102BE100906ECBF0A3F0A37401F0755706201A077D
:102BF1007E457FEB124046906FDEE004F0C2121278
:042C01000026C210D7
:012C050022AC
:104E3300E559602CE4906CB2F0A3E559F0906EB69E
:104E4300E0906CB4F0A37419F0906EDE63A201904D
:104E53006CB663A201AF5912337EE4F5597F012288
:034E63007F0022AB
:0B501100302905C2297F01227F002208
:0100210022BC
:06503600E4F559F54522E6
:0A501C00E4906941F0A3F0A3F02234
:104E66002043616E457247495400200A004572721C
:104E76004C656E43616E21000A002043616E4572E7
:0F4E860072434821000A20526571457272210063
:103BEB00E59B541F6020201A1A7E4E7F66124046BA
:103BFB00E59B541FFF7E007D031241277E4E7F7095
:103C0B00124046E4F59BE5BA30E010E4F5B375B12C
:103C1B0080F5B2D22BF556906FF5F0E5CFF470032B
:103C2B00023D40752901E4F528E5CFF455297003D1
:103C3B00023D2EE528C454F0F5B1E5B2547F642063
:103C4B006003023CFFE5B3540FF54B85BC47E5BD64
:103C5B00541FFF131313541FFFE5BD54E044184FBB
:103C6B00F548E5BDC43354E0FFE5BE131313541FF1
:103C7B004FF549E5BEC43354E0FFE5BF13131354AE
:103C8B001F4FF54A85A34C85A34D85A34E85A34FA6
:103C9B0085A35085A35185A35285A353E4F5B22088
:103CAB00010CE547547EB5470575B350800375B3DA
:103CBB00D0E54B700AE547547EB547037F002230B1
:103CCB000108E54730E7037F0022E54BD39408401A
:103CDB001D201A177E4E7F73124046AF4B7E007D20
:103CEB00031241277E4E7F7E1240467F0022E54B1A
:103CFB002405FF22E5B2549F6023201A207E4E7FBD
:103D0B0080124046AFB27E007D03124127AFB37ED7
:103D1B00007D031241277E4E7F7E124046E4F5B2B2
:103D2B0075B3D0E52925E0F5290528E528C39408C6
:073D3B005003023C347F003D
:013D4200225E
:104B3C00906EDDE0C39464505675B180E4F5B3F526
:104B4C00B28547BCE549C4135407FFE54854E04F10
:104B5C00F5BDE54933333354F8FFE54AC413540724
:104B6C004FF5BEE54A33333354F8F5BF854CA38576
:104B7C004DA3854EA3854FA38550A38551A3855284
:104B8C00A38553A3E54B540F2450F5B375560AC2B5
:024B9C002B22CA
:104B9E0075B190E5B220E613201A107E4E7F8B126F
:104BAE004046AFB27E007D03124127E4F5B3F5B265
:104BBE0074872513F582E43461F583E0F5BCE4F5E2
:104BCE00BD74882513F582E43461F583E0FF333339
:104BDE003354F8F5BE75BF78051305137487251386
:104BEE00F582E43461F583E07002F51375B350225B
:09502600EF6003C29622D296222B
:104A740043AB01C2E8C2EAE4FFEFC454F0F5B1C3AA
:104A8400EF64809488500575B3D08003E4F5B3E4F3
:104A9400F5B2F5BCF5BDF5BEF5BFF5C4F5C5F5C673
:104AA400F5C7F5A3F5A3F5A3F5A3F5A3F5A3F5A31E
:104AB400F5A30FBF0EC3906EDDE0FF25E0F5B475DE
:104AC400B50C75B66C75A11275AB0275C13E75C394
:044AD400FF75C203A5
:014AD80022BB
:101142005452414E5A004D415842005254530044A9
:10115200454C4159004D4F4445004B5000545500F9
:1011620043414E004B5654004154004449520043FF
:10117200414E4D4F4E00475254494D45005449543B
:1011820053005453494E5600003E2A2C312CCFE0D6
:10119200F0E0ECE5F2F0FB20F3EFF0E0E2EBFFFE33
:1011A200F9E5E3EE20EAEEEDF2F0EEEBEBE5F0E04E
:1011B20020CACF20C8F1E5F2FC0A003E4C2C6B306D
:1011C200312C25732C43EAEEF0EEF1F2FC20EDE037
:1011D20020F8E8EDE52043414E2C30202D2035301B
:1011E20030EAE1283530EC292C31202D203530EA47
:1011F200E128353030EC290A0030202D20353030FE
:10120200EAE1283530EC290031202D203530EAE1A1
:1012120028353030EC29003E532C6B30322C2562BD
:10122200752CCCE0EAF12E20E0E4F0E5F120E1EBD0
:10123200EEEAE020D2D128302D38290A003E532C84
:101242006B30332C2562752CCCE0EAF12E20E0E4E1
:10125200F0E5F120E1EBEEEAE020D2C8D228302D11
:1012620038290A003E532C6B30342C2562752CCC65
:10127200E0EAF12E20E0E4F0E5F120E1EBEEEAE035
:1012820020D2D328302D38290A003E422C63303137
:101292002C2562752CC2F2EEF0E8F7EDFBE920EAAC
:1012A200EEEDF2F0EEEBEBE5F020EDE020F8E8ED0C
:1012B200E50A003E2A2C312CCFE0F0E0ECE5F2F01A
:1012C200FB20EFF0EEF2EEEAEEEBE020C3F0E0ED11
:1012D200E8F220EFEE20EFEEF0F2F3205253323339
:1012E200320A003E432C61636B2C25732CCFEEF047
:1012F200FFE4EEEA20C0D4C10A00312DD2D1283059
:101302002B312920322DD2C8D228302920332DD298
:10131200D320342DD2C8D228312920352DD2D1283C
:10132200322B332920382DD2C8C8003E4C2C6B30CA
:10133200352C256C752CD1EAEEF0EEF1F2FC20EEA4
:10134200E1ECE5EDE020EDE020EFEEF0F2F32C3100
:1013520030302C3230302C3330302C3630302C318F
:101362003230302C323430302C343830302C393664
:1013720030302C31393230302C33383430302C3557
:10138200373630302C3131353230300A003E532C72
:101392006B30362C2562752CCDEEECE5F020CACFF1
:1013A200200A003E422C6730312C2562752CCCE09D
:1013B200E3E8F1F2F0E0EBFC0A003E422C67303247
:1013C2002C2562752CC8EDE2E5F0F2E8F0EEE2E0E1
:1013D200F2FC20E7EDE0F7E5EDE8FF20D2D10A00CC
:1013E2003E422C6730332C2562752CC7E0EFF0E0CB
:1013F200F8E8E2E0F2FC20E2F0E5ECFF20F1E5F0B3
:10140200E2E5F0E00A003E422C6730342C2562759A
:101412002CC2FBF1F2E0E2EBFFF2FC20525453202B
:10142200EFF0E820EFE5F0E5E4E0F7E50A003E53EF
:101432002C6730352C2562752CC7E0E4E5F0E6EA2E
:10144200E020EFE5F0E5E4E0F7E820EFEEF1EBE590
:101452002052545320282A3130ECF1290A003C2131
:10146200003C6B30313D003C6B30323D003C6B3018
:10147200333D003C6B30343D003C6330313D003C39
:101482006B30353D003C6B30363D003C6730313DC2
:10149200003C6730323D003C6730333D003C6730F2
:1014A200343D003C6730353D000ACFE5F0E5E4E02D
:1014B200F7E03A2000544949204379636C650A00F9
:1014C2005453204379636C650A0054530A0054490B
:1014D200540A005455204F4B0A0054552044696168
:1014E200670A005455205265710A00205455205451
:1014F200696D654F5554210A000ACFF0E8E5EC3AD0
:1015020020000A4352432045525221000AD7F3E6F3
:10151200EEE920EDEEECE5F020CACF21000A52659B
:101522007154533120000A52657154533520000A18
:1015320052657154495420000ACFF0E8EDFFF2E001
:1015420020EAEEECE0EDE4E020D2D320002020D22D
:10155200D320E7E0EDFFF2EE210A000ACDE520EF0D
:10156200EEEDFFEB20F2E8EF20EFE0EAE5F2E0211A
:101572000A0000112332465765748C9DAFBECADB48
:10158200E9F810013322564775649C8DBFAEDACB61
:10159200F9E82130021367764455ADBC8E9FEBFA11
:1015A200C8D93120120377665445BDAC9E8FFBEA41
:1015B200D8C94253617004152736CEDFEDFC8899F5
:1015C200ABBA5243716014053726DECFFDEC988921
:1015D200BBAA6372405125340617EFFECCDDA9B8D1
:1015E2008A9B7362504135241607FFEEDCCDB9A801
:1015F2009A8B8495A7B6C2D3E1F008192B3A4E5FB5
:101602006D7C9485B7A6D2C3F1E018093B2A5E4FE0
:101612007D6CA5B48697E3F2C0D129380A1B6F7E90
:101622004C5DB5A49687F3E2D0C139281A0B7F6EC0
:101632005C4DC6D7E5F48091A3B24A5B69780C1D74
:101642002F3ED6C7F5E49081B3A25A4B79681C0DA0
:101652003F2EE7F6C4D5A1B082936B7A48592D3C50
:101662000E1FF7E6D4C5B1A092837B6A58493D2C80
:101672001E0F0089129B24AD36BF48C15AD36CE5B8
:101682007EF78108931AA52CB73EC940DB52ED6460
:10169200FF76028B109926AF34BD4AC358D16EE74C
:1016A2007CF5830A9118A72EB53CCB42D950EF6640
:1016B200FD74048D169F20A932BB4CC55ED768E12C
:1016C2007AF3850C971EA128B33ACD44DF56E96020
:1016D200FB72068F149D22AB30B94EC75CD56AE30C
:1016E20078F1870E951CA32AB138CF46DD54EB6200
:1016F200F97008811A932CA53EB740C952DB64EDFC
:1017020076FF89009B12AD24BF36C148D35AE56CDF
:10171200F77E0A8318912EA73CB542CB50D966EFCB
:1017220074FD8B029910AF26BD34C34AD158E76EBF
:10173200F57C0C851E9728A13AB344CD56DF60E9AB
:1017420072FB8D049F16A920BB32C54CD75EE1689F
:10175200F37A0E871C952AA338B146CF54DD62EB8B
:1017620070F98F069D14AB22B930C74ED55CE36A7F
:10177200F1780008040C020A060E0109050D030B9C
:10178200070FFF1142FF1148FF114DFF1151FF11C9
:1017920057FF115CFF115FFF1162FF1166FF116AB3
:1017A200FF116DFF1171FF1178FF117FFF1184FF8F
:0217B200118A9A
:104FDA00EF540F90177493FEC454F0FEEFC4540FAD
:044FEA00932EFF22E1
:030023000244CDC7
:0B44CD00C0E0C083C082C0D075D018D2
:1044D800309852C298755E01AF9920064820020BA9
:1044E800EF64027040D202D291803A300A04C20AC4
:1044F8008024BF0904D20A802CBF0205530B808098
:1045080024BF0312906614E50BF0630B80530B80F5
:10451800C202C291800F7437250BF582E43466F528
:1045280083EFF0050B30992B300326906185E0FF6F
:10453800E50CC39F4008C203D20DC2908013D290ED
:10454800AF0C050C74372FF582E43467F583E0F57A
:0345580099C2996C
:09455B00D0D0D082D083D0E03230
:103D43007BFF7A11798B122381906EDDE0701475FD
:103D53002FFF7530117531FB7BFF7A1179BD12236B
:103D6300818012752FFF75301275310A7BFF7A112E
:103D730079BD1223817BFF7A127919906186E0F570
:103D83002F1223817BFF7A12793F906101E0F52F97
:103D93001223817BFF7A127966906100E0F52F127E
:103DA30023817BFF7A12798CA201E433F52F12234E
:103DB300817BFF7A1279B5122381752FFF7530123B
:103DC3007531FC7BFF7A1279E5122381906838E024
:103DD300FEA3E0FFC3E49FFFE49EFEAB07FA339527
:103DE300E0F9F87F007E8C7D0A7C001227528F3227
:103DF3008E318D308C2F7BFF7A13792D1223817BAB
:103E0300FF7A13798F906403E0F52F1223817BFFF0
:103E13007A1379A5A20EE4336401F52F1223817B73
:103E2300FF7A1379BCA209E433F52F1223817BFFB8
:103E33007A1379E2A204E433F52F1223817BFF7A0C
:103E4300147908A20BE433F52F1223817BFF7A1434
:093E5300793085092F1223812228
:103916007E147F6012467EEF4E70037F0122E49094
:103926006EDDF07E147F6312467EEF4E6015124FF9
:1039360093BF3106906EDD740AF0BF3206906EDDDD
:103946007464F07E147F6912467EEF4E600A124B55
:10395600FE906186EFF080069061867402F07E1418
:103966007F6F12467EEF4E600A124BFE906101EFAA
:10397600F080069061017402F07E147F7512467E17
:10398600EF4E600A124BFE906100EFF080069061E8
:10399600007402F07E147F7B12467EEF4E600D129D
:1039A6004BFEEC4D4E4F24FF92018002C2017E1465
:1039B6007F8112467EEF4E6023124BFEA804A905B6
:1039C600AA06AB077F007E8C7D0A7C001227521266
:1039D60027E4906838EEF0A3EFF0800A9068387418
:1039E600FFF0A374DCF07E147F8712467EEF4E60F4
:1039F6000A124BFE906403EFF08006906403740194
:103A0600F07E147F8D12467EEF4E600E124F93EFBE
:103A160024D0640124FF920E8002C20E7E147F938E
:103A260012467EEF4E600C124F93EF24D024FF9285
:103A3600098002C2097E147F9912467EEF4E600C01
:103A4600124F93EF24D024FF92048002C2047E1406
:103A56007F9F12467EEF4E600C124F93EF24D024C8
:103A6600FF920B8002C20B7E147FA512467EEF4E9C
:0E3A76006007124BFE8F098003E4F5097F0004
:013A8400221F
:102EA700E4F527E52775F003A42484F582E43417B5
:102EB700F583E493FB740193FA740293F912267B6A
:102EC70070030230AFE4F529F52AF528746925283F
:102ED700F582E43469F583E0FF70030230AAE52741
:102EE70075F003A42484F582E43417F583E493FB97
:102EF700740193FA740293F9852982758300122667
:102F070094FEEFB50608752A0105290230A5E52AC2
:102F170070030230A5EE60030230A0E527B40F006E
:102F270040030230AA902F33F8282873022F60023B
:102F37002FA7022FE0022FE50230AA02303D023010
:102F4700AA0230100230AA0230AA02306A02309474
:102F57000230980230AA02309C74692528F9E434BB
:102F670069FA7B01C0031B8B32753300753400E4AB
:102F7700F535D0031235FD8F2E8E2D8D2C8C2BAB76
:102F87002EAA2DA92CA82B7F007E8C7D0A7C0012EF
:102F970027521227E4906838EEF0A3EFF00230AA28
:102FA70074692528F582E43469F583E024D09061BB
:102FB70086F0746A2528F582E43469F583E024D025
:102FC700906101F0746B2528F582E43469F583E09C
:102FD70024D0906100F00230AAD20B0230AA7469A3
:102FE7002528F9E43469FA7B01C0031B8B3275335A
:102FF70000753400E4F535D0031235FD8F2E8E2D84
:103007008D2C8C2B8F090230AA74692528F9E4349A
:1030170069FA7B01C0031B8B32753300753400E4FA
:10302700F535D0031235FD8F2E8E2D8D2C8C2B90E0
:103037006EDDEFF0806D74692528F9E43469FA7B59
:1030470001C0031B8B32753300753400E4F535D0AE
:10305700031235FD8F2E8E2D8D2C8C2B906403EF54
:10306700F0804074692528F9E43469FA7B01C003CC
:103077001B8B32753300753400E4F535D0031235F8
:10308700FD8F2E8E2D8D2C8C2BD20E8016D201808B
:1030970012D204800EC209800AE4F52AF529052810
:0830A700022ED30527022EAA18
:0130AF0022FE
:10345500C228C20CC208C207C205E4906837F0C290
:103465000F9066167405F0C22AE4F508FF7F4090B8
:1034750061B9E4F0A3DFFCE4FF7F20906617E4F078
:10348500A3DFFCE4FF74042FF582E43466F583E4DE
:10349500F0740C2FF582E43466F583E4F00FBF0871
:1034A500E4E4F50DF50EF512F511906302F0906365
:1034B50001F0C203C20DC206C202C20AF50C906138
:1034C50085F0F509F50BF55EC200C20B90683874FE
:1034D500FFF0A374F4F0E4906403F0C20EC201C2DD
:1034E50004D209906EDDF0123916EF6003122EA793
:1034F500E4F5137E617F87906186E0F513E513C3DC
:1035050094014007E513D394084003E4F513E5134C
:1035150060220FEFAC0670010E14F5828C8374C423
:10352500F015130FEFAC0670010E14F5828C83E5D0
:1035350013F080DA906101E0F513E513C3940140BF
:1035450007E513D394084003E4F513E51360220F50
:10355500EFAC0670010E14F5828C8374C8F0151358
:103565000FEFAC0670010E14F5828C83E513F08025
:10357500DA906100E0F513E513C394014007E51304
:10358500D394084003E4F513E51360220FEFAC066E
:1035950070010E14F5828C8374C2F015130FEFAC15
:1035A5000670010E14F5828C83E513F080DA0FEFB7
:1035B500AC0670010E14F5828C83E4F08F828E8345
:1035C500F0F513C2ADF5C9D2CDD2CCC2C9C2CAF588
:1035D500CDF5CC906838E0F5CBA3E0F5CA85CBCD29
:1035E50085CACCD29ED29CD2CAC2ACC298C29975A9
:0735F500B81075B710D2AC4D
:0135FC0022AC
:104FEE00E5106FFF90167493650FF510EF90157422
:034FFE0093F50F19
:01500100228C
:0242D5008F2D2B
:1042D700E4FC752E61752F02F510F50FFDEDC39502
:1042E7002D5017052FE52FAE2E7002052E14F582DF
:1042F7008E83E0FF124FEE0D80E3052FE52FAE2EE4
:104307007002052E14F5828E83E510F0852F8285C5
:104317002E83E50FF0052D052D7E677F37752E61FE
:10432700752F028F828E837402F00FBF00010E0C6F
:10433700E4FDEDC3952D5038852F82852E83E0F956
:1043470064026008E964036003B9090D8F828E83F4
:104357007409F00FBF00010E0C8F828E83E9F00FF6
:10436700BF00010E0C052FE52F7002052E0D80C230
:0F4377008F828E837403F00FBF00010E0CAF0412
:014386002214
:03503C00C2062287
:104D87008F2C20033AAF2C1242D5906185EFF0208B
:104D97001A127E147FAB1240467E617F02E4FBADA0
:104DA7002C124201300B057F01125026E5096003E2
:104DB700F55B22E4F50CD203C2992099FDD2992222
:022C06008F2815
:102C0800E54724BE7003022E4F24FA7003022DC933
:102C180024046003022EA6E54830E703022CCD30D9
:102C28001B077E147FB7124046E54A6068E549C332
:102C380094024003022EA6E5497007E54A14F529D7
:102C48008006E54A241FF529E52975F004A4240324
:102C5800F582746335F0F5837D4C7F0412336CE59F
:102C68002975F004A42401F582746235F0F5837D9A
:102C7800507F0412336C74F92549F582E43461F508
:102C8800837481F074B92529F582E43461F583747D
:102C980001F0D20722301B077E147FC2124046740F
:102CA800042549F582E43466F5837401F0E5497535
:102CB800F004A42417F582746635F0F5837D4C7F03
:102CC8000412336C22E54B64086003022EA6E54922
:102CD800C394044003022EA6301B077E147FCC1237
:102CE8004046752801E54A5407FFE528A8070880EB
:102CF80002C333D8FCF5287408250EF50EB50D0669
:102D08007408250DF50DE54A547FFFE549C4335491
:102D1800E02FFE7400250EF582E43460F583EEF0B2
:102D2800E54AC394805022EF131313541FFFE5495B
:102D380025E025E02F2417F582E43466F583E0FFCB
:102D4800E528F4FEEF5EF0802EE54A547FFF13136A
:102D580013541FFFE54925E025E02F2417F582E4E9
:102D68003466F583E04528F07400250EF582E434D6
:102D780060F583E04480F07401250EF582E4346048
:102D8800F5837D4C7F0412336CE551FEE550FF7CE2
:102D9800007D0A1226C1EF7405250EF582E4346021
:102DA800F583EFF07406250EF582E43460F583E5CB
:102DB80052F07407250EF582E43460F583E553F08C
:102DC80022301B077E147FD0124046E54A54E06447
:102DD800407003022EA6E549701DE54A1313543FBF
:102DE800FF7401A807088002C333D8FC421190631E
:102DF80001E04511F08024E54964016003022EA634
:102E0800E54A1313543FFF7401A807088002C3332F
:102E1800D8FC4212906302E04512F0E54975F020B3
:102E2800A4FFE54A547F7C002FFFEC35F0FEEF2528
:102E3800E0FFEE33FE74042FF58274643EF5837D63
:102E48004CAF4B12336C22E54AB40113301B077E9A
:102E5800147FD5124046E54D04906FF6F0C228E580
:102E68004AB40216240CF582E43466F583E54DF085
:102E7800301B077E147FDC124046E54AB4031F244A
:102E88000CF582E43466F583E54DF0301B077E14BB
:0E2E98007FE5124046302806906FDE7402F08F
:012EA6002209
:10002600906403E070030208E630102F050A90661C
:1000360016E0600214F0906837E0600214F0C21017
:10004600302818906184E004F0E0D3940A400C3024
:100056001B077E147FED124046C228E55BB4010EF5
:10006600E4F55BF50CD203C2992099FDD2993003D1
:100076000DE50AD394064009C203D20D8003E4F5C8
:100086000A300D0AC20D300B05E4FF12502630036C
:1000960003020542E55B6003020542200E062005C9
:1000A60003020542C205300F29C20FE4906102F037
:1000B600A37408F0906403E0906104F0906615E084
:1000C600906105F0A374FEF0A3748FF07F06124DC5
:1000D6008722906FF6E0FF6025E4906102F0A3743A
:1000E60008F0906403E0906104F0A37483F0A3EF3A
:1000F600F0E4A3F0906FF6F07F06124D8722E50E2E
:10010600650D7003020205906837E060030202DFA6
:10011600E50D2408F528E4906102F0A37408F09038
:100126006403E0906104F0A374F0F0A37406F0A3F6
:100136007491F074062528F582E43460F583E09026
:100146006108F074072528F582E43460F583E090B1
:100156006109F074012528F582E43460F583E090A6
:10016600610AF074022528F582E43460F583E09094
:10017600610BF074032528F582E43460F583E09082
:10018600610CF074042528F582E43460F583E09070
:10019600610DF074002528F582E43460F583E0FFF4
:1001A600547FFEC39440500BEFC454F00490610E8C
:1001B600F0801674002528F582E43460F583E0FFAC
:1001C600C454F0240590610EF074002528F582E4ED
:1001D6003460F583E0FFEEC4540F90610FF0EF54E6
:1001E60080FF74052528F582E43460F583E02F90BE
:1001F6006110F09068377414F07F0F124D8722302B
:10020600086AE4906102F0A37408F0906403E09039
:100216006104F0A37441F0A37420F0752A61752B74
:1002260007E4F52874172528F582E43466F583E09B
:10023600F529300906FF124FDA8F29852B82852A88
:1002460083E529F0F4FFE5822408F582E43583F599
:1002560083EFF0052BE52B7002052A0528E528C358
:10026600940840C07F15124D87C20822300C6AE4FC
:10027600906102F0A37408F0906403E0906104F0CA
:10028600A37445F0A37420F0752A61752B077528B1
:100296000874172528F582E43466F583E0F52930DD
:1002A6000906FF124FDA8F29852B82852A83E529D5
:1002B600F0F4FFE5822408F582E43583F583EFF058
:1002C600052BE52B7002052A0528E528C394104066
:1002D600C07F15124D87C20C222007030203E2904D
:1002E60061FAE0FF9061F9E04F5401D394005003A6
:1002F6000203E2E4F52874B92528F582E43461F5B1
:1003060083E070030203D474B92528F582E43461CE
:10031600F583E4F0906102F0A37408F0906403E0C2
:10032600906104F0A374F0F0A37403F0A37491F049
:10033600E528C4540F2408A3F0E528540FA3F0E5DC
:100346002825E025E0F5282401F582E43462F583CA
:10035600E090610AF074022528F582E43462F583A0
:10036600E090610BF074032528F582E43462F5838E
:10037600E090610CF074042528F582E43462F5837C
:10038600E090610DF0E4A3F074032528F582E434CF
:1003960063F583E090610FF074042528F582E43458
:1003A60063F583E0906110F074052528F582E43446
:1003B60063F583E0906111F074062528F582E43434
:1003C60063F583E0906112F07F11124D87220528B4
:1003D600E528C3944050030202FCC207906616E06B
:1003E600704130043E7478F0E4906102F0A3740822
:1003F600F0906403E0906104F0A374F0F0E4A3F0DD
:10040600A37490F0A37408F0E4A3F0A3F0A3F0A300
:10041600F0A3F0A3F0A3F0A3F0A3F0A3F07F1112D2
:100426004D8722E508C39404506FE50825E0FF7464
:1004360003A807088002C333D8FCF52855116528A0
:100446007053E528F45211E4906102F0A37408F0A9
:10045600906403E0906104F0A374F0F0A37402F0DA
:10046600A37491F0E5082420A3F0E5083333335450
:10047600F875F002A42404F582E5F03464F583638C
:10048600A20190610963A2017F1012337E7F1712C9
:100496004D870508220508808AE508C3940850762A
:1004A600E50824FC25E0FF7403A807088002C3338F
:1004B600D8FCF528551265287058E528F45212E440
:1004C600906102F0A37408F0906403E0906104F078
:1004D600A374F0F0A37402F0A37491F0E50854033A
:1004E6002440A3F0E50833333354F875F002A4240E
:1004F60004F582E5F03464F58363A2019061096333
:10050600A2017F1012337E7F17124D87050853080C
:10051600072205088083E4F508200E20E490610296
:10052600F0A37408F0906403E0906104F0A3749063
:10053600F0E4A3F0A3F07F06124D8722906614E044
:10054600FF70030208E6F529E4F0201A1F7E147FE7
:10055600FB124046E52954802437F582E43466AF21
:1005660082FEE529547FFDE4FB124201E529700372
:100576000208E6E5295480FF2437F582E43466ADA7
:1005860082F52A8D2BE4F510F50F8F28E528C39503
:10059600295018052BE52BAE2A7002052A14F58280
:1005A6008E83E0FF124FEE052880E1E50F451060CF
:1005B6000E301A030208E67E157F0412404622E535
:1005C6002954802437F582E43466AF82F52A8F2BCE
:1005D6007402252BF52BE4352AF52A852B82F58323
:1005E600E0FF906403E0FEEF6E600E301A0302082F
:1005F600E67E157F0E12404622052BE52B7002057E
:100606002AF582852A83E0FFB43003D20522EF64FF
:100616000170030208E6EF64187037906605E0FF84
:10062600906604E04F600CD208201A077E157F1FE3
:10063600124046906607E0FF906606E04F700302A0
:1006460008E6D20C301A030208E67E157F2812400F
:100656004622852B82852A83E0B41915201A077E47
:10066600157F31124046906301E0F511A3E0F512C3
:1006760022852B82852A83E0FF54F064F060030212
:10068600076E906615EFF0052BE52B7002052AF52F
:1006960082852A83E0FF64807033052BE52B700288
:1006A600052AF582852A83E0644060030208E6D2C3
:1006B6000F052BE52B7002052AF582852A83E06457
:1006C6000860030208E6D204906616F022EFB40131
:1006D60027052BE52B7002052AF582852A83E0641F
:1006E6004F60030208E6906837E070030208E6747C
:1006F60008250DF50DE4F022852B82852A83E0601E
:10070600030208E6052BE52B7002052AF582852AE9
:1007160083E0644260030208E6052BE52B700205C0
:100726002AF582852A83E0906FE0F0052BE52B7091
:1007360002052AF582852A83E0906FE1F0052BE514
:100746002B7002052AF582852A83E0906FE2F00578
:100756002BE52B7002052AF582852A83E0906FE34C
:10076600F0D22AC204D20F22852B82852A83E0FF8B
:1007760064116008EF641260030208C4E529547F1F
:10078600640E60030208C4201A077E157F3A1240E1
:100796004630280E301A030208E67E157F4F1240B7
:1007A6004622852B82852A83E0540314F529052BDE
:1007B600E52B7002052AF582852A83E0F52830E7C5
:1007C60009E4906FDFF0906FE4F0E52830E60BE483
:1007D600906FDFF0906FE47410F0E52830E50B9031
:1007E6006FDF7401F0E4906FE4F0E52830E40C90DC
:1007F6006FDF7401F0906FE47410F0E52830E30BBE
:10080600906FDF7402F0E4906FE4F0E52830E20CBC
:10081600906FDF7402F0906FE47410F0E52830E119
:100826000B906FDF7403F0E4906FE4F0E52830E09E
:100836000C906FDF7403F0906FE47410F07402256F
:100846002BF52BE4352AF52A852B82F583E0F5284E
:1008560030E700E52830E607906FE4E02402F0E593
:100866002830E507906FE4E02404F0E52830E4073B
:10087600906FE4E02406F0E52830E307906FE4E0AB
:100886002408F0E52830E207906FE4E0240AF0E55A
:100896002830E107906FE4E0240CF0E52830E0070B
:1008A600906FE4E0240EF0906FE4E02529F0D22862
:1008B600E4906184F0906FDEF0906FF6F022201ADB
:1008C6001F7E157F5D124046E52954802437F58248
:1008D600E43466AF82FEE529547FFDE4FB12420153
:0108E60022EF
:1045FE000217B4E493A3F8E493A34003F68001F208
:10460E0008DFF48029E493A3F85407240CC8C333BD
:10461E00C4540F4420C8834004F456800146F6DF8C
:10462E00E4800B010204081020408090502FE47E9D
:10463E00019360BCA3FF543F30E509541FFEE49381
:10464E00A360010ECF54C025E060A840B8E493A348
:10465E00FAE493A3F8E493A3C8C582C8CAC583CA73
:10466E00F0A3C8C582C8CAC583CADFE9DEE780BE2B
:01503500007A
:10267B00BB010689828A83E0225002E722BBFE025D
:09268B00E32289828A83E4932290
:10269400BB010CE58229F582E5833AF583E02250FB
:1026A40006E92582F8E622BBFE06E92582F8E22245
:0D26B400E58229F582E5833AF583E493225F
:1026C100BC000BBE0029EF8DF084FFADF022E4CCFD
:1026D100F875F008EF2FFFEE33FEEC33FCEE9DECC6
:1026E100984005FCEE9DFE0FD5F0E9E4CEFD22ED0C
:1026F100F8F5F0EE8420D21CFEADF075F008EF2F56
:10270100FFED33FD4007985006D5F0F222C398FD46
:052711000FD5F0EA22E3
:1027160075F008758200EF2FFFEE33FECD33CDCC7A
:1027260033CCC58233C5829BED9AEC99E5829840FD
:102736000CF582EE9BFEED9AFDEC99FC0FD5F0D6DA
:10274600E4CEFBE4CDFAE4CCF9A88222B800C1B904
:102756000059BA002DEC8BF084CFCECDFCE5F0CB42
:10276600F97818EF2FFFEE33FEED33FDEC33FCEB7B
:1027760033FB10D703994004EB99FB0FD8E5E4F936
:10278600FA227818EF2FFFEE33FEED33FDEC33FC23
:10279600C933C910D7059BE99A4007EC9BFCE99A17
:1027A600F90FD8E0E4C9FAE4CCFB2275F010EF2F5C
:1027B600FFEE33FEED33FDCC33CCC833C810D7075C
:1027C6009BEC9AE899400AED9BFDEC9AFCE899F897
:0E27D6000FD5F0DAE4CDFBE4CCFAE4C8F9222A
:0E27E400C3E49FFFE49EFEE49DFDE49CFC2206
:1027F200EB9FF5F0EA9E42F0E99D42F0E89C45F03D
:0128020022B3
:0C280300ECF0A3EDF0A3EEF0A3EFF02248
:10280F00A8828583F0D083D0821228261228261220
:10281F002826122826E473E493A3C583C5F0C58345
:10282F00C8C582C8F0A3C583C5F0C583C8C582C813
:01283F002276
:10231F00E53B242FF8E6053B22782C302602782F58
:10232F00E475F0011228A102267B201FEB7F2ED22D
:10233F001F8018EF540F2490D43440D4FF30230B58
:10234F00EF24BFB41A0050032461FFE53C6002156F
:10235F003C053FE53F7002053E30260D782CE475B5
:10236F00F0011228A1EF022840024CB47403D226C8
:10237F008003E4C226F53B8B2C8A2D892EE4F53C95
:10238F00F53EF53FE53C60077F2012235A80F57537
:10239F003DFFC220C21FC221C222C224C225C227B2
:1023AF00122328FF700D3026057F0012236BAF3FDD
:1023BF00AE3E22B4255FC2D5C223122328FF24D0FC
:1023CF00B40A00501A75F00A783C30D50508B6FFEC
:1023DF000106C6A426F620D5047002D22280D92485
:1023EF00CFB41A00EF5004C2E5D22302256BD220DE
:1023FF0080C6D21F80C0D22180BCD2D580BAD22451
:10240F0080B47F2012235A2021077401B53C00406D
:10241F00F112231FFF12235A022393D227D22580B2
:10242F009512231FFB12231FFA12231FF94A4B7019
:10243F0006793C7A267BFF20212EE53C602A7E0020
:10244F008E8275830012269460060EEE653D70F045
:10245F00C2D5EBC0E0EAC0E0E9C0E0EE1225B2D091
:10246F00E0F9D0E0FAD0E0FB12267BFF60AAEBC0C8
:10247F00E0EAC0E0E9C0E012235AD0E02401F9D02D
:10248F00E03400FAD0E0FBE53D0460DCD53DD980B7
:10249F00877BFF7A2579AED221809C7910800279D3
:1024AF0008C225C2278008D2D5790A8004790AC2CA
:1024BF00D5E53D047002F53DE4FAFDFEFF12231F42
:1024CF00FC7B0820201312231FFD7B10301F0A12E4
:1024DF00231FFE12231FFF7B20EC3382D592D55092
:1024EF0013C3E4301F069FFFE49EFEE42020039DEC
:1024FF00FDE49CFCE4CBF8C220EC700CCFCECDCC2D
:10250F00E824F8F870F38017C3EF33FFEE33FEEDD6
:10251F0033FDEC33FCEB33FB994002FB0FD8E9EBB7
:10252F00302005F8D0E0C448B220C0E00AEC4D4E90
:10253F004F78207B0070C2EAB53D0040BCC0E0126E
:10254F0025B4D0F0D0E0202004C4C0E0C4B220C035
:10255F00F0122343D0F0D5F0EB022393122900247D
:10256F00305324AA5824014C23FD4224AE4F24B6E5
:0F257F004424B64924164324BC5524A04624A066
:10258E004524A047265C5024052D24092E242C2BEF
:10259E00240D23242A2026452A23C548000024245E
:1025AE003F3F3F00790AA2D5202214302409B910EA
:1025BE00020404B9080104A2D5202502500104200A
:1025CE0021689221B53C005034C0E07F20302219A2
:1025DE007F30A22172257224500F12260BC221C207
:1025EE0025C224C2277F30800F302403E9C0E012B9
:1025FE00235A302403D0E0F9D0E0B53CCC30241778
:10260E007F30B9100C12235A7F583023077F788001
:10261E0003B9080312235A3021057F2D02235A7F56
:10262E00202027F87F2B2025F322922180CF286EA1
:10263E00756C6C2900D22012231F3020F8C220782E
:10264E003C30D50108F60223C52D504349581223BC
:10265E001F2403B405004001E49026579312234B28
:0D266E00743A12234BD222753C040224AAB8
:1035FD008B2F8A308931E4F53BF53AF539F538F5FD
:10360D0036F537E533453445326012EBC0E0EAC09C
:10361D00E0E9C0E0AB32AA33A9341228B1AB2F05D3
:10362D0031E531AA307002053014F912267BF53CD4
:10363D00C394094007E53CD3940D40E1E53C64207B
:10364D0060DBE53CB42D054337038016E53CB42B18
:10365D0005433701800C74FF2531F53174FF35308A
:10366D00F530E53560046410703FAB2FAA30A931F9
:10367D0012267B64306009E535702E75350A802978
:10368D00900001122694FF64786004EFB458134340
:10369D00370175351074022531F531E43530F530CB
:1036AD008007E5357003753508AB2F0531E531AA77
:1036BD00307002053014F912267BF53CC39461403D
:1036CD000AE53CD3947A5003533CDF74D0253CF586
:1036DD003CC3940A400CE53C9411406D74F9253CB3
:1036ED00F53CE53CD395355060433701853B40852E
:1036FD003A3F85393E85383DAF357E00E4FCFDAB64
:10370D003BAA3AA939A838122852C8ECC8C9EDC944
:10371D00CAEECACBEFCBE4FCFDFEEB253CF53BEE50
:10372D003AF53AED39F539EC38F538AF3BAE3AADFF
:10373D0039FCAB40AA3FA93EA83DD31227F2500356
:10374D000236B64337040236B6E53720E003E4808F
:10375D002DE53345344532601EAB2FE53124FFF99D
:10376D00E53034FFFAEBC0E0EAC0E0E9C0E0AB328F
:10377D00AA33A9341228B1E53730E20774FFFFFEF2
:10378D00FDFC22E537AF3BAE3AAD39AC3830E10345
:04379D000227E422F9
:10284000BB010689828A83F0225002F722BBFE0177
:02285000F32271
:10285200E88FF0A4CC8BF0A42CFCE98EF0A42CFC25
:102862008AF0EDA42CFCEA8EF0A4CDA8F08BF0A4A3
:102872002DCC3825F0FDE98FF0A42CCD35F0FCEB02
:102882008EF0A4FEA9F0EB8FF0A4CFC5F02ECD39C7
:0F289200FEE43CFCEAA42DCE35F0FDE43CFC2234
:1028A100FAE6FB0808E6F925F0F618E6CA3AF62238
:1028B100BB011A89828A83D0F0D0E0F8D0E0F9D048
:1028C100E0FAD0E0FBE8C0E0C0F002292F5016E9A1
:1028D100F8D083D082D0E0F9D0E0FAD0E0FBC0821A
:1028E100C083022926BBFE16E9F8D083D082D0E04E
:0F28F100F9D0E0FAD0E0FBC082C0830229382280
:10290000D083D082F8E4937012740193700DA3A366
:1029100093F8740193F5828883E47374029368607A
:06292000EFA3A3A380DF7A
:09292600EBF608EAF608E9F622D6
:09292F00EBF0A3EAF0A3E9F022A9
:09293800EBF208EAF208E9F222D0
:00000001FF
